:100000000C9434000C9451000C9451000C94510049
:100010000C9451000C9451000C9451000C9451001C
:100020000C9451000C9451000C9451000C94380124
:100030000C9451000C9451000C9451000C945100FC
:100040000C9451000C9451000C9451000C945100EC
:100050000C9451000C9451000C9451000C945100DC
:100060000C9451000C94510011241FBECFEFD8E026
:10007000DEBFCDBF11E0A0E0B1E0EEE2F6E002C0ED
:1000800005900D92AA30B107D9F721E0AAE0B1E0BE
:1000900001C01D92AC30B207E1F70E94E5020C945A
:1000A00015030C94000084B18F6184B985B18FEF82
:1000B00085B92FEF85EA9EE0215080409040E1F71E
:1000C00000C0000085B115B80895092E000CAA0BD8
:1000D000BB0B9C01AD0184E0220F331F441F551F51
:1000E0008A95D1F760E074E284EF90E00E94F30219
:1000F000215031093093C5002093C40088E18093DA
:10010000C10086E08093C200E0ECF0E080818D7F4A
:10011000808308959091C00095FFFCCF8093C60026
:1001200008958091C00087FFFCCF8091C60008959C
:10013000EAE7F0E0808187608083ACE7B0E08C91F3
:1001400080648C938C918F778C938C918F7D8C9322
:10015000ABE7B0E08C91887F8C938081806880834E
:10016000808180648083089590917C00982B909387
:100170007C0090917A00906490937A0090917A003C
:1001800096FDFCCF90917C008095892380937C0024
:1001900080917800909179000895E1E8F0E0808105
:1001A0008860808380818460808380818160808397
:1001B00088E690E09093890080938800EFE6F0E075
:1001C00080818260808308958AB18AB98BB18FEF74
:1001D0008BB984B18F6384B9089580E0D1E0C9B14F
:1001E000C2FBCC27C0F9CD274B9BC2604C9BC4609F
:1001F0004D9BC8604E9BC061C81719F08C2F0E94A0
:100200008A008FE39CE90197F1F700C000008C2F72
:10021000E6CFC0E080E00E94B4008C0181E00E9443
:10022000B400C1110BC0C80134E0969587953A958A
:10023000E1F780680E948A00C1E009C024E0969539
:1002400087952A95E1F7806C0E948A00C0E08FE3D1
:100250009CE90197F1F700C00000DCCF0E949100FB
:1002600085B98FE39CE90197F1F700C00000F6CF54
:100270001F920F920FB60F9211242F933F934F931B
:100280005F936F937F938F939F93AF93BF93EF93FE
:10029000FF9380910A0181110CC081E080930A01D3
:1002A000789480910001909101019EBF8DBF0E94C2
:1002B0002E01813009F036C00F920FB6F8940F92DC
:1002C0001F9211242F923F924F925F926F927F92D2
:1002D0008F929F92AF92BF92CF92DF92EF92FF9256
:1002E0000F931F932F933F934F935F936F937F933E
:1002F0008F939F93AF93BF93CF93DF93EF93FF932E
:100300008DB79EB7909301018093000182E08093A6
:100310000A01789480910301909104019EBF8DBFE2
:100320000E940901823009F036C00F920FB6F8948E
:100330000F921F9211242F923F924F925F926F92D1
:100340007F928F929F92AF92BF92CF92DF92EF9265
:10035000FF920F931F932F933F934F935F936F934E
:100360007F938F939F93AF93BF93CF93DF93EF933D
:10037000FF938DB79EB7909304018093030183E0B0
:1003800080930A01789480910601909107019EBFA5
:100390008DBF0E94ED0080910B01811154C00F921E
:1003A0000FB6F8940F921F9211242F923F924F9202
:1003B0005F926F927F928F929F92AF92BF92CF92F5
:1003C000DF92EF92FF920F931F932F933F934F93E0
:1003D0005F936F937F938F939F93AF93BF93CF93CD
:1003E000DF93EF93FF938DB79EB7909307018093B0
:1003F000060180910001909101019EBF8DBFFF9188
:10040000EF91DF91CF91BF91AF919F918F917F91AC
:100410006F915F914F913F912F911F910F91FF909D
:10042000EF90DF90CF90BF90AF909F908F907F9094
:100430006F905F904F903F902F901F900F900FBE46
:100440000F9081E056C0813009F056C00F920FB670
:10045000F8940F921F9211242F923F924F925F9225
:100460006F927F928F929F92AF92BF92CF92DF92C4
:10047000EF92FF920F931F932F933F934F935F93AE
:100480006F937F938F939F93AF93BF93CF93DF939C
:10049000EF93FF938DB79EB7909301018093000176
:1004A00080910301909104019EBF8DBFFF91EF9158
:1004B000DF91CF91BF91AF919F918F917F916F917C
:1004C0005F914F913F912F911F910F91FF90EF906E
:1004D000DF90CF90BF90AF909F908F907F906F9064
:1004E0005F904F903F902F901F900F900FBE0F90F6
:1004F00082E080930B0157C0823009F054C00F9204
:100500000FB6F8940F921F9211242F923F924F92A0
:100510005F926F927F928F929F92AF92BF92CF9293
:10052000DF92EF92FF920F931F932F933F934F937E
:100530005F936F937F938F939F93AF93BF93CF936B
:10054000DF93EF93FF938DB79EB790930401809351
:10055000030180910601909107019EBF8DBFFF911D
:10056000EF91DF91CF91BF91AF919F918F917F914B
:100570006F915F914F913F912F911F910F91FF903C
:10058000EF90DF90CF90BF90AF909F908F907F9033
:100590006F905F904F903F902F901F900F900FBEE5
:1005A0000F9010920B017894FF91EF91BF91AF9152
:1005B0009F918F917F916F915F914F913F912F917B
:1005C0000F900FBE0F901F9018950E94530080E867
:1005D00095E20E9465000E9498000E94CD000E9452
:1005E000E4007894FFCFA1E21A2EAA1BBB1BFD01E9
:1005F0000DC0AA1FBB1FEE1FFF1FA217B307E40702
:10060000F50720F0A21BB30BE40BF50B661F771F59
:10061000881F991F1A9469F7609570958095909539
:0E0620009B01AC01BD01CF010895F894FFCFFE
:0A062E0000070000050000030000B3
:00000001FF
